:0200000480007A
:100000006F000005732F2034930F80006308FF03F7
:10001000930F90006304FF03930FB0006300FF038E
:10002000130F000063040F0067000F00732F2034CC
:1000300063540F006F00400093E19153171F0000BD
:1000400023223FFC171F000023200FFC6FF01FFF2F
:100050009300000013010000930100001302000050
:100060009302000013030000930300001304000038
:100070009304000013050000930500001306000020
:100080009306000013070000930700001308000008
:10009000930800001309000093090000130A0000F0
:1000A000930A0000130B0000930B0000130C0000D8
:1000B000930C0000130D0000930D0000130E0000C0
:1000C000930E0000130F0000930F0000732540F102
:1000D0006310050097020000938202017390523072
:1000E000735044749702000093820201739052305F
:1000F00073500018970200009382420273905230AE
:100100009B021000939252039382F2FF7390023B82
:100110009302F0017390023A73504030970200004E
:1001200093824201739052307350203073503030BC
:100130009301000097020000938202ED7390523009
:10014000130510001315F501635C05000F00F00F97
:10015000930110009308D005130500007300000000
:1001600093020000638A020073905210B7B200003D
:100170009B8292107390223073500030372500001C
:1001800073200530735030009702000093824201C3
:1001900073901234732540F17300203093012000D6
:1001A000370501001B0505C0530505F4531505E48B
:1001B00093031000631C750E9301300037C50000D7
:1001C0001B0505C0530505F4531505E493032000F2
:1001D000631E750C93014000378500001B05F53F39
:1001E000530505F4531505E4930340006310750CA3
:1001F0009301500037850000530505F4531505E4BD
:10020000930380006314750A9301600013050000D6
:10021000530505F4531505E49303000163187508AD
:10022000930170001305F03F530505F4531505E4E1
:1002300093030002631C750693018000374500009C
:100240001B0505C0530505F4531505E4930300048D
:10025000631E750493019000378500001B0505C0DF
:10026000530505F4531505E4930300086310750462
:100270009301A000378500001B0515C0530505F448
:10028000531505E493030010631275029301B00047
:10029000378500001B0505E0530505F4531505E4FB
:1002A0009303002063147500631030020F00F00FF9
:1002B000638001009391110093E111009308D00530
:1002C00013850100730000000F00F00F9301100070
:1002D0009308D0051305000073000000731000C0E0
:1002E000000000000000000000000000000000000E
:0C02F00000000000000000000000000002
:1010000000000000000000000000000000000000E0
:1010100000000000000000000000000000000000D0
:1010200000000000000000000000000000000000C0
:1010300000000000000000000000000000000000B0
:081040000000000000000000A8
:040000058000000077
:00000001FF
